******************************************************************************
               TMS320C6x Linker PC v7.4.10                     
******************************************************************************
>> Linked Thu Feb 23 20:04:03 2017

OUTPUT FILE NAME:   <GPIO.out>
ENTRY POINT SYMBOL: "_c_int00"  address: 1080d0a0


MEMORY CONFIGURATION

         name            origin    length      used     unused   attr    fill
----------------------  --------  ---------  --------  --------  ----  --------
  MSMC_RAM              0c000000   00200000  00000000  00200000  RWIX
  VECTORS               10800000   00000200  00000200  00000000  RWIX
  LL2_RW_DATA           10800200   0003fe00  000117ac  0002e654  RWIX
  DDR3_CODE             80000000   01000000  00000000  01000000  RWIX
  DDR3_R_DATA           81000000   01000000  00000000  01000000  RWIX
  DDR3_RW_DATA          82000000   06000000  00000000  06000000  RWIX


SEGMENT ALLOCATION MAP

run origin  load origin   length   init length attrs members
----------  ----------- ---------- ----------- ----- -------
10800000    10800000    0000f378   0000f378    r-x
  10800000    10800000    00000200   00000200    r-x vecs
  10800200    10800200    0000d4c0   0000d4c0    r-x .text
  1080d6c0    1080d6c0    00001cb8   00001cb8    r-- .const
1080f378    1080f378    00001800   00000000    rw-
  1080f378    1080f378    00001000   00000000    rw- .stack
  10810378    10810378    00000800   00000000    rw- .sysmem
10810b78    10810b78    00000950   00000830    rw-
  10810b78    10810b78    00000648   00000648    rw- .fardata
  108111c0    108111c0    000001e8   000001e8    rw- .far
  108113a8    108113a8    00000120   00000000    rw- .cio
108114c8    108114c8    000000a8   000000a8    rw-
  108114c8    108114c8    000000a8   000000a8    rw- .neardata
10811570    10811570    0000043c   0000043c    r--
  10811570    10811570    0000043c   0000043c    r-- .cinit


SECTION ALLOCATION MAP

 output                                  attributes/
section   page    origin      length       input sections
--------  ----  ----------  ----------   ----------------
vecs       0    10800000    00000200     
                  10800000    00000200     GPIO_vectors.obj (vecs)

.text      0    10800200    0000d4c0     
                  10800200    00005c20     K2_common.obj (.text)
                  10805e20    000006a0     GPIO_main.obj (.text:retain)
                  108064c0    00000600     K2_common.obj (.text:retain)
                  10806ac0    000005c0     rts6600_elf.lib : divd.obj (.text:__c6xabi_divd)
                  10807080    000005c0                     : _printfi.obj (.text:_getarg_diouxp)
                  10807640    00000520                     : _printfi.obj (.text:_setfield)
                  10807b60    00000460                     : _printfi.obj (.text:_printfi)
                  10807fc0    00000440     K2_common.obj (.text:Core_MPAX)
                  10808400    00000400     GPIO_main.obj (.text)
                  10808800    000003a0     rts6600_elf.lib : fputs.obj (.text:fputs)
                  10808ba0    00000320                     : _printfi.obj (.text:_pproc_fge)
                  10808ec0    000002e0                     : _printfi.obj (.text:_pproc_fwp)
                  108091a0    000002a0                     : _printfi.obj (.text:fcvt)
                  10809440    00000280                     : divf.obj (.text:__c6xabi_divf)
                  108096c0    00000280                     : _printfi.obj (.text:ecvt)
                  10809940    00000280                     : memory.obj (.text:free)
                  10809bc0    00000240                     : imath64.obj (.text:__c6xabi_divull)
                  10809e00    00000240                     : _printfi.obj (.text:_pconv_e)
                  1080a040    00000240                     : _printfi.obj (.text:_pproc_diouxp)
                  1080a280    00000220                     : _printfi.obj (.text:_pproc_str)
                  1080a4a0    00000220                     : fputc.obj (.text:fputc)
                  1080a6c0    00000200                     : _printfi.obj (.text:_pconv_g)
                  1080a8c0    00000200                     : setvbuf.obj (.text:setvbuf)
                  1080aac0    000001c0                     : _printfi.obj (.text:_mcpy)
                  1080ac80    000001a0                     : trgdrv.obj (.text:HOSTrename)
                  1080ae20    000001a0                     : imath40.obj (.text:__c6xabi_divul)
                  1080afc0    00000180                     : copy_decompress_rle.obj (.text:__TI_decompress_rle_core)
                  1080b140    00000180                     : memory.obj (.text:malloc)
                  1080b2c0    00000140                     : _printfi.obj (.text:_pproc_fflags)
                  1080b400    00000140                     : lowlev.obj (.text:getdevice)
                  1080b540    00000120                     : fclose.obj (.text:_closefile)
                  1080b660    00000120                     : _printfi.obj (.text:_ltostr)
                  1080b780    00000120                     : fseek.obj (.text:fseek)
                  1080b8a0    00000100                     : trgdrv.obj (.text:HOSTlseek)
                  1080b9a0    00000100                     : autoinit.obj (.text:_auto_init_elf)
                  1080baa0    00000100                     : _io_perm.obj (.text:_wrt_ok)
                  1080bba0    00000100                     : cpy_tbl.obj (.text:copy_in)
                  1080bca0    000000e0                     : trgdrv.obj (.text:HOSTopen)
                  1080bd80    000000e0                     : trgdrv.obj (.text:HOSTread)
                  1080be60    000000e0                     : _printfi.obj (.text:_div)
                  1080bf40    000000e0                     : atoi.obj (.text:atoi)
                  1080c020    000000e0                     : lowlev.obj (.text:close)
                  1080c100    000000e0                     : ltoa.obj (.text:ltoa)
                  1080c1e0    000000e0                     : memset.obj (.text:memset)
                  1080c2c0    000000e0                     : printf.obj (.text:printf)
                  1080c3a0    000000c0                     : trgdrv.obj (.text:HOSTunlink)
                  1080c460    000000c0                     : trgdrv.obj (.text:HOSTwrite)
                  1080c520    000000c0                     : divu.obj (.text:__divu)
                  1080c5e0    000000c0                     : fflush.obj (.text:_doflush)
                  1080c6a0    000000c0                     : exit.obj (.text:exit)
                  1080c760    000000c0                     : tls.obj (.text:tls:init:__TI_tls_init)
                  1080c820    000000a0                     : trgdrv.obj (.text:HOSTclose)
                  1080c8c0    000000a0                     : fopen.obj (.text:_cleanup)
                  1080c960    000000a0                     : _printfi.obj (.text:_ecpy)
                  1080ca00    000000a0                     : _printfi.obj (.text:_fcpy)
                  1080caa0    000000a0                     : memory.obj (.text:_minit)
                  1080cb40    000000a0                     : _printfi.obj (.text:_pconv_f)
                  1080cbe0    000000a0                     : lowlev.obj (.text:finddevice)
                  1080cc80    000000a0                     : lowlev.obj (.text:lseek)
                  1080cd20    000000a0                     : memcpy64.obj (.text:memcpy)
                  1080cdc0    000000a0                     : memory.obj (.text:minsert)
                  1080ce60    000000a0                     : memory.obj (.text:mremove)
                  1080cf00    000000a0                     : lowlev.obj (.text:write)
                  1080cfa0    00000080                     : fixfu.obj (.text:__c6xabi_fixfu)
                  1080d020    00000080                     : llshift.obj (.text:__c6xabi_llshl)
                  1080d0a0    00000080                     : boot.obj (.text:_c_int00)
                  1080d120    00000080                     : trgmsg.obj (.text:readmsg)
                  1080d1a0    00000080                     : lowlev.obj (.text:unlink)
                  1080d220    00000060                     : cpp_init.obj (.text:__TI_cpp_init)
                  1080d280    00000060                     : frcmpyd_div.obj (.text:__c6xabi_frcmpyd_div)
                  1080d2e0    00000060                     : llshift.obj (.text:__c6xabi_llshru)
                  1080d340    00000060                     : imath64.obj (.text:_subcull)
                  1080d3a0    00000060                     : memccpy.obj (.text:memccpy)
                  1080d400    00000060                     : trgmsg.obj (.text:writemsg)
                  1080d460    00000040     GPIO_vectors.obj (.text)
                  1080d4a0    00000040     rts6600_elf.lib : isinf.obj (.text:__c6xabi_isinf)
                  1080d4e0    00000040                     : _printfi.obj (.text:__c6xabi_isnan)
                  1080d520    00000040                     : strasg.obj (.text:__strasgi_64plus)
                  1080d560    00000040                     : args_main.obj (.text:_args_main)
                  1080d5a0    00000040                     : fputs.obj (.text:puts)
                  1080d5e0    00000020                     : negll.obj (.text:__c6xabi_negll)
                  1080d600    00000020                     : _lock.obj (.text:_nop)
                  1080d620    00000020                     : printf.obj (.text:_outc)
                  1080d640    00000020                     : printf.obj (.text:_outs)
                  1080d660    00000020                     : exit.obj (.text:abort)
                  1080d680    00000020                     : copy_decompress_none.obj (.text:decompress:none:__TI_decompress_none)
                  1080d6a0    00000020                     : copy_decompress_rle.obj (.text:decompress:rle24:__TI_decompress_rle24)

.const     0    1080d6c0    00001cb8     
                  1080d6c0    00001b38     K2_common.obj (.const:.string)
                  1080f1f8    00000101     rts6600_elf.lib : ctype.obj (.const:.string:_ctypes_)
                  1080f2f9    00000002                     : fputs.obj (.const:.string)
                  1080f2fb    00000001     --HOLE-- [fill = 0]
                  1080f2fc    00000038     GPIO_main.obj (.const:.string)
                  1080f334    00000023     rts6600_elf.lib : _printfi.obj (.const:.string)
                  1080f357    00000001     --HOLE-- [fill = 0]
                  1080f358    00000020     K2_common.obj (.const:$P$T0$1)

.stack     0    1080f378    00001000     UNINITIALIZED
                  1080f378    00000008     rts6600_elf.lib : boot.obj (.stack)
                  1080f380    00000ff8     --HOLE--

.sysmem    0    10810378    00000800     UNINITIALIZED
                  10810378    00000008     rts6600_elf.lib : memory.obj (.sysmem)
                  10810380    000007f8     --HOLE--

.fardata   0    10810b78    00000648     
                  10810b78    000001e0     rts6600_elf.lib : defs.obj (.fardata:_ftable)
                  10810d58    000000a0                     : lowlev.obj (.fardata:_stream)
                  10810df8    00000078                     : lowlev.obj (.fardata:_device)
                  10810e70    00000078     K2_common.obj (.fardata:gstruMpuAddrRange)
                  10810ee8    0000005c     K2_common.obj (.fardata:gCIC_exception_events)
                  10810f44    00000004     rts6600_elf.lib : defs.obj (.fardata)
                  10810f48    00000050     K2_common.obj (.fardata:gpTimerRegs)
                  10810f98    00000040     K2_common.obj (.fardata:gCIC_EXC_EN_MASK)
                  10810fd8    00000040     K2_common.obj (.fardata:gpMPU_regs)
                  10811018    00000038     K2_common.obj (.fardata:gpEDMA_TC_regs)
                  10811050    00000024     K2_common.obj (.fardata:input_clk_str)
                  10811074    00000004     --HOLE--
                  10811078    00000024     K2_common.obj (.fardata:internal_exception_str)
                  1081109c    00000004     --HOLE--
                  108110a0    00000020     K2_common.obj (.fardata:K2E_boot_mode_str)
                  108110c0    00000020     K2_common.obj (.fardata:K2H_K2K_boot_mode_str)
                  108110e0    00000020     K2_common.obj (.fardata:K2L_boot_mode_str)
                  10811100    00000020     K2_common.obj (.fardata:bus_err_stat_str)
                  10811120    00000020     GPIO_main.obj (.fardata:usaCIC_GPIO_INT_table)
                  10811140    00000018     K2_common.obj (.fardata:Peri_MPU_err_type_str)
                  10811158    00000014     K2_common.obj (.fardata:gpEDMA_CC_regs)
                  1081116c    00000004     --HOLE--
                  10811170    00000010     K2_common.obj (.fardata:device_type_str)
                  10811180    0000000c     rts6600_elf.lib : exit.obj (.fardata)
                  1081118c    0000000c                     : memory.obj (.fardata)
                  10811198    00000008     K2_common.obj (.fardata:Ns_str)
                  108111a0    00000008     K2_common.obj (.fardata:boot_master_str)
                  108111a8    00000008     K2_common.obj (.fardata:endian_str)
                  108111b0    00000008     K2_common.obj (.fardata:gpDDR3ControlRegs)
                  108111b8    00000008     rts6600_elf.lib : _lock.obj (.fardata)

.far       0    108111c0    000001e8     
                  108111c0    00000140     rts6600_elf.lib : defs.obj (.far) [fill = 0]
                  10811300    00000090     K2_common.obj (.far) [fill = 0]
                  10811390    00000010     K2_common.obj (.far:Core_MPAX)
                  108113a0    00000008     rts6600_elf.lib : trgdrv.obj (.far) [fill = 0]

.cio       0    108113a8    00000120     UNINITIALIZED
                  108113a8    00000120     rts6600_elf.lib : trgmsg.obj (.cio)

.neardata 
*          0    108114c8    000000a8     
                  108114c8    000000a0     K2_common.obj (.neardata)
                  10811568    00000008     GPIO_main.obj (.neardata)

.cinit     0    10811570    0000043c     
                  10811570    00000357     (.cinit..fardata.load) [load image, compression = rle]
                  108118c7    00000001     --HOLE-- [fill = 0]
                  108118c8    000000a8     (.cinit..neardata.load) [load image, compression = rle]
                  10811970    0000001a     (.cinit..far.load) [load image, compression = rle]
                  1081198a    00000002     --HOLE-- [fill = 0]
                  1081198c    00000008     (__TI_handler_table)
                  10811994    00000018     (__TI_cinit_table)

.rodata    0    10811570    00000000     UNINITIALIZED

.bss       0    10811570    00000000     UNINITIALIZED


LINKER GENERATED COPY TABLES

__TI_cinit_table @ 10811994 records: 3, size/record: 8, table size: 24
	.fardata: load addr=10811570, load size=00000357 bytes, run addr=10810b78, run size=00000648 bytes, compression=rle
	.neardata: load addr=108118c8, load size=000000a8 bytes, run addr=108114c8, run size=000000a8 bytes, compression=rle
	.far: load addr=10811970, load size=0000001a bytes, run addr=108111c0, run size=000001e8 bytes, compression=rle


LINKER GENERATED HANDLER TABLE

__TI_handler_table @ 1081198c records: 2, size/record: 4, table size: 8
	index: 0, handler: __TI_decompress_rle24
	index: 1, handler: __TI_decompress_none


GLOBAL SYMBOLS: SORTED ALPHABETICALLY BY Name 

address    name
--------   ----
10804d68   Bus_error_handler
1080d660   C$$EXIT
1080d458   C$$IO$$
10805908   CPU_interrupt_enable
10805860   CPU_interrupt_init
10804e44   DDR3_IRQ_handler
10802b98   EDMA_CC_error_handler
10802dac   EDMA_TC_error_handler
10801ce4   EDMA_TC_priority_cfg
10801c60   EDMA_channel_TC_cfg
1080252c   EDMA_copy
10802ed8   EDMA_error_handler
10802324   EDMA_event_disable
108022b4   EDMA_event_enable
10802738   EDMA_fill
10801d4c   EDMA_init
10802400   EDMA_interrupt_disable
10802390   EDMA_interrupt_enable
1080246c   EDMA_wait
10805830   EXC_NMI
10805770   EXC_internal
10805848   EXC_swgen
108064c0   Exception_service_routine
108061d8   GPIO_16_up_ISR
10806008   GPIO_8_12_ISR
10805e20   GPIO_ISR
10808534   GPIO_Interrupts_Init
1080864c   GPIO_init
108086d4   GPIO_loopback_test
10808798   GPIO_print_interrupt_status
1080c820   HOSTclose
1080b8a0   HOSTlseek
1080bca0   HOSTopen
1080bd80   HOSTread
1080ac80   HOSTrename
1080c3a0   HOSTunlink
1080c460   HOSTwrite
10802b00   IDMA_copy
10802ad4   IDMA_wait
108110a0   K2E_boot_mode_str
108110c0   K2H_K2K_boot_mode_str
108110e0   K2L_boot_mode_str
10801c18   K2_ARM_LPSC_eanble
10801214   K2_ARM_PLL_init
108012d4   K2_PASS_PLL_init
10803834   K2_SMS_MPAX_init
10805d68   K2_common_device_init
10805a48   K2_get_device_info
108059f8   K2_get_device_speed_grade
10805940   K2_lookup_device_speed_grade
10805058   KeyStone_CIC_EXC_handler
10804a6c   KeyStone_CIC_exception_events_mapping
10803418   KeyStone_CorePac_AID_map
108052b0   KeyStone_EXC_external
10804b84   KeyStone_Exception_cfg
10808150   KeyStone_MPAX_seg_setup
10803d98   KeyStone_MPU_MPPA_modify
10803e84   KeyStone_MPU_interrupt_enable
10803f38   KeyStone_MPU_interrupts_enable
10803b20   KeyStone_MPU_range_setup
10803ba4   KeyStone_MPU_setup
108038a8   KeyStone_MSMC_MP_interrupt_en
10804154   KeyStone_MSMC_RAM_EDC_enable
10804794   KeyStone_MSMC_RAM_EDC_handler
10804214   KeyStone_MSMC_RAM_EDC_interrupt_en
10803a30   KeyStone_MSMC_protection_exception_handler
1080108c   KeyStone_PLL_init
108034a8   KeyStone_PrivID_Remap
10803524   KeyStone_SES_MPAX_seg_delete
10803730   KeyStone_SES_MPAX_setup
108035a8   KeyStone_SMS_MPAX_seg_delete
1080362c   KeyStone_SMS_MPAX_setup
10808304   KeyStone_XMC_MPAX_setup
10805dd4   KeyStone_common_CPU_init
10801b68   KeyStone_disable_PSC_Power_Domain
10801ab4   KeyStone_disable_PSC_module
10801968   KeyStone_enable_PSC_module
10800bf4   KeyStone_main_PLL_init
10804074   KeyStone_peripherals_MPU_excepiton_handler
10803f78   KeyStone_peripherals_MPU_fault_status
1080316c   L1D_memory_protection_cfg
108043b8   L1P_EDC_setup
10804670   L1P_ED_handler
108030d8   L1P_memory_protection_cfg
10803034   L1_MPPA_setup
10803200   L1_cache_protection
10811554   LL2_EDC_DMA_err_str
10811558   LL2_EDC_L1D_err_str
1081155c   LL2_EDC_L1P_err_str
10804440   LL2_EDC_handler
10804304   LL2_EDC_scrub
1080426c   LL2_EDC_setup
10811550   LL2_EDC_victim_err_str
10803210   LL2_MPPA_setup
108032ac   LL2_Memory_Protection_cfg
10806870   Nested_Exception_service_routine
10811198   Ns_str
10811140   Peri_MPU_err_type_str
10801518   Reset_Timer
10801924   Service_Watchdog
108013e0   TSC_delay_ms
10801478   TSC_delay_us
108013cc   TSC_init
10801568   Timer64_Init
108113a8   __CIOBUF_
10811994   __TI_CINIT_Base
108119ac   __TI_CINIT_Limit
1081198c   __TI_Handler_Table_Base
10811994   __TI_Handler_Table_Limit
UNDEFED    __TI_INITARRAY_Base
UNDEFED    __TI_INITARRAY_Limit
10810378   __TI_STACK_END
00001000   __TI_STACK_SIZE
108114c8   __TI_STATIC_BASE
00000800   __TI_SYSMEM_SIZE
UNDEFED    __TI_TLS_INIT_Base
UNDEFED    __TI_TLS_INIT_Limit
00000001   __TI_args_main
1080d220   __TI_cpp_init
1080d680   __TI_decompress_none
1080d6a0   __TI_decompress_rle24
10811188   __TI_enable_exit_profile_output
ffffffff   __TI_pprof_out_hndl
ffffffff   __TI_prof_data_size
ffffffff   __TI_prof_data_start
1080c760   __TI_tls_init
ffffffff   __binit__
10806ac0   __c6xabi_divd
10809440   __c6xabi_divf
1080c520   __c6xabi_divu
1080ae20   __c6xabi_divul
10809bc0   __c6xabi_divull
1080cfa0   __c6xabi_fixfu
1080d280   __c6xabi_frcmpyd_div
1080d4a0   __c6xabi_isinf
1080d020   __c6xabi_llshl
1080d2e0   __c6xabi_llshru
1080d5e0   __c6xabi_negll
1080d520   __c6xabi_strasgi_64plus
ffffffff   __c_args__
1080c520   __divu
1080d520   __strasgi_64plus
1080d560   _args_main
1080b9a0   _auto_init_elf
1080d0a0   _c_int00
1080c8c0   _cleanup
10811180   _cleanup_ptr
1080b540   _closefile
1080f1f8   _ctypes_
1080c5e0   _doflush
10811184   _dtors_ptr
10810f44   _ft_end
10810b78   _ftable
108111b8   _lock
1080caa0   _minit
1080d600   _nop
10807b60   _printfi
1080f378   _stack
1080d340   _subcull
10810378   _sys_memory
108111c0   _tmpnams
108111bc   _unlock
1080baa0   _wrt_ok
1080d660   abort
1080bf40   atoi
ffffffff   binit
108111a0   boot_master_str
10811100   bus_err_stat_str
10801374   calc_cycle_measure_overhead
108086a0   check_GPIO
1080c020   close
1080bba0   copy_in
10811548   cycle_measure_overhead
10811170   device_type_str
108111a8   endian_str
10811300   exception_record
1080c6a0   exit
1080a4a0   fputc
10808800   fputs
10809940   free
1080b780   fseek
10811540   gARM_Core_Speed_Hz
10810f98   gCIC_EXC_EN_MASK
10811564   gCIC_EXC_out_num
10810ee8   gCIC_exception_events
10811544   gMain_Core_Speed_Hz
108114e4   gpARM_regs
108114d0   gpBootCfgRegs
108114cc   gpCGEM_regs
108114e8   gpCIC0_regs
108114ec   gpCIC1_regs
108114f0   gpCIC_regs
108111b0   gpDDR3ControlRegs
108114f4   gpEDMA_CC0_regs
108114f8   gpEDMA_CC1_regs
108114fc   gpEDMA_CC2_regs
10811500   gpEDMA_CC3_regs
10811504   gpEDMA_CC4_regs
10811158   gpEDMA_CC_regs
10811508   gpEDMA_TC_0_0_regs
1081150c   gpEDMA_TC_0_1_regs
10811510   gpEDMA_TC_1_0_regs
10811514   gpEDMA_TC_1_1_regs
10811518   gpEDMA_TC_1_2_regs
1081151c   gpEDMA_TC_1_3_regs
10811520   gpEDMA_TC_2_0_regs
10811524   gpEDMA_TC_2_1_regs
10811528   gpEDMA_TC_2_2_regs
1081152c   gpEDMA_TC_2_3_regs
10811530   gpEDMA_TC_3_0_regs
10811534   gpEDMA_TC_3_1_regs
10811538   gpEDMA_TC_4_0_regs
1081153c   gpEDMA_TC_4_1_regs
10811018   gpEDMA_TC_regs
108114e0   gpGPIO_regs
10810fd8   gpMPU_regs
108114dc   gpMSMC_regs
108114d4   gpPLLC_regs
108114d8   gpPSC_regs
10810f48   gpTimerRegs
108114c8   gpXMC_regs
10810e70   gstruMpuAddrRange
10811560   guwIntcCICExcEvtIdx
10811050   input_clk_str
10811078   internal_exception_str
10807fc0   lock_mem_prot_regs
1080cc80   lseek
1080c100   ltoa
10808758   main
1080b140   malloc
10811390   mem_prot_key
1080d3a0   memccpy
1080cd20   memcpy
10803910   memory_protection_exception_handler
1080c1e0   memset
10811568   num_GPIO
1080c2c0   printf
1080d5a0   puts
1080d120   readmsg
1080d1a0   remove
1080a8c0   setvbuf
1081156c   uiGPIO_host_event_num
1081154c   uiLL2_scrub_addr
1080d1a0   unlink
10808088   unlock_mem_prot_regs
10811120   usaCIC_GPIO_INT_table
10800000   vectors
1080cf00   write
1080d400   writemsg


GLOBAL SYMBOLS: SORTED BY Symbol Address 

address    name
--------   ----
00000001   __TI_args_main
00000800   __TI_SYSMEM_SIZE
00001000   __TI_STACK_SIZE
10800000   vectors
10800bf4   KeyStone_main_PLL_init
1080108c   KeyStone_PLL_init
10801214   K2_ARM_PLL_init
108012d4   K2_PASS_PLL_init
10801374   calc_cycle_measure_overhead
108013cc   TSC_init
108013e0   TSC_delay_ms
10801478   TSC_delay_us
10801518   Reset_Timer
10801568   Timer64_Init
10801924   Service_Watchdog
10801968   KeyStone_enable_PSC_module
10801ab4   KeyStone_disable_PSC_module
10801b68   KeyStone_disable_PSC_Power_Domain
10801c18   K2_ARM_LPSC_eanble
10801c60   EDMA_channel_TC_cfg
10801ce4   EDMA_TC_priority_cfg
10801d4c   EDMA_init
108022b4   EDMA_event_enable
10802324   EDMA_event_disable
10802390   EDMA_interrupt_enable
10802400   EDMA_interrupt_disable
1080246c   EDMA_wait
1080252c   EDMA_copy
10802738   EDMA_fill
10802ad4   IDMA_wait
10802b00   IDMA_copy
10802b98   EDMA_CC_error_handler
10802dac   EDMA_TC_error_handler
10802ed8   EDMA_error_handler
10803034   L1_MPPA_setup
108030d8   L1P_memory_protection_cfg
1080316c   L1D_memory_protection_cfg
10803200   L1_cache_protection
10803210   LL2_MPPA_setup
108032ac   LL2_Memory_Protection_cfg
10803418   KeyStone_CorePac_AID_map
108034a8   KeyStone_PrivID_Remap
10803524   KeyStone_SES_MPAX_seg_delete
108035a8   KeyStone_SMS_MPAX_seg_delete
1080362c   KeyStone_SMS_MPAX_setup
10803730   KeyStone_SES_MPAX_setup
10803834   K2_SMS_MPAX_init
108038a8   KeyStone_MSMC_MP_interrupt_en
10803910   memory_protection_exception_handler
10803a30   KeyStone_MSMC_protection_exception_handler
10803b20   KeyStone_MPU_range_setup
10803ba4   KeyStone_MPU_setup
10803d98   KeyStone_MPU_MPPA_modify
10803e84   KeyStone_MPU_interrupt_enable
10803f38   KeyStone_MPU_interrupts_enable
10803f78   KeyStone_peripherals_MPU_fault_status
10804074   KeyStone_peripherals_MPU_excepiton_handler
10804154   KeyStone_MSMC_RAM_EDC_enable
10804214   KeyStone_MSMC_RAM_EDC_interrupt_en
1080426c   LL2_EDC_setup
10804304   LL2_EDC_scrub
108043b8   L1P_EDC_setup
10804440   LL2_EDC_handler
10804670   L1P_ED_handler
10804794   KeyStone_MSMC_RAM_EDC_handler
10804a6c   KeyStone_CIC_exception_events_mapping
10804b84   KeyStone_Exception_cfg
10804d68   Bus_error_handler
10804e44   DDR3_IRQ_handler
10805058   KeyStone_CIC_EXC_handler
108052b0   KeyStone_EXC_external
10805770   EXC_internal
10805830   EXC_NMI
10805848   EXC_swgen
10805860   CPU_interrupt_init
10805908   CPU_interrupt_enable
10805940   K2_lookup_device_speed_grade
108059f8   K2_get_device_speed_grade
10805a48   K2_get_device_info
10805d68   K2_common_device_init
10805dd4   KeyStone_common_CPU_init
10805e20   GPIO_ISR
10806008   GPIO_8_12_ISR
108061d8   GPIO_16_up_ISR
108064c0   Exception_service_routine
10806870   Nested_Exception_service_routine
10806ac0   __c6xabi_divd
10807b60   _printfi
10807fc0   lock_mem_prot_regs
10808088   unlock_mem_prot_regs
10808150   KeyStone_MPAX_seg_setup
10808304   KeyStone_XMC_MPAX_setup
10808534   GPIO_Interrupts_Init
1080864c   GPIO_init
108086a0   check_GPIO
108086d4   GPIO_loopback_test
10808758   main
10808798   GPIO_print_interrupt_status
10808800   fputs
10809440   __c6xabi_divf
10809940   free
10809bc0   __c6xabi_divull
1080a4a0   fputc
1080a8c0   setvbuf
1080ac80   HOSTrename
1080ae20   __c6xabi_divul
1080b140   malloc
1080b540   _closefile
1080b780   fseek
1080b8a0   HOSTlseek
1080b9a0   _auto_init_elf
1080baa0   _wrt_ok
1080bba0   copy_in
1080bca0   HOSTopen
1080bd80   HOSTread
1080bf40   atoi
1080c020   close
1080c100   ltoa
1080c1e0   memset
1080c2c0   printf
1080c3a0   HOSTunlink
1080c460   HOSTwrite
1080c520   __c6xabi_divu
1080c520   __divu
1080c5e0   _doflush
1080c6a0   exit
1080c760   __TI_tls_init
1080c820   HOSTclose
1080c8c0   _cleanup
1080caa0   _minit
1080cc80   lseek
1080cd20   memcpy
1080cf00   write
1080cfa0   __c6xabi_fixfu
1080d020   __c6xabi_llshl
1080d0a0   _c_int00
1080d120   readmsg
1080d1a0   remove
1080d1a0   unlink
1080d220   __TI_cpp_init
1080d280   __c6xabi_frcmpyd_div
1080d2e0   __c6xabi_llshru
1080d340   _subcull
1080d3a0   memccpy
1080d400   writemsg
1080d458   C$$IO$$
1080d4a0   __c6xabi_isinf
1080d520   __c6xabi_strasgi_64plus
1080d520   __strasgi_64plus
1080d560   _args_main
1080d5a0   puts
1080d5e0   __c6xabi_negll
1080d600   _nop
1080d660   C$$EXIT
1080d660   abort
1080d680   __TI_decompress_none
1080d6a0   __TI_decompress_rle24
1080f1f8   _ctypes_
1080f378   _stack
10810378   __TI_STACK_END
10810378   _sys_memory
10810b78   _ftable
10810e70   gstruMpuAddrRange
10810ee8   gCIC_exception_events
10810f44   _ft_end
10810f48   gpTimerRegs
10810f98   gCIC_EXC_EN_MASK
10810fd8   gpMPU_regs
10811018   gpEDMA_TC_regs
10811050   input_clk_str
10811078   internal_exception_str
108110a0   K2E_boot_mode_str
108110c0   K2H_K2K_boot_mode_str
108110e0   K2L_boot_mode_str
10811100   bus_err_stat_str
10811120   usaCIC_GPIO_INT_table
10811140   Peri_MPU_err_type_str
10811158   gpEDMA_CC_regs
10811170   device_type_str
10811180   _cleanup_ptr
10811184   _dtors_ptr
10811188   __TI_enable_exit_profile_output
10811198   Ns_str
108111a0   boot_master_str
108111a8   endian_str
108111b0   gpDDR3ControlRegs
108111b8   _lock
108111bc   _unlock
108111c0   _tmpnams
10811300   exception_record
10811390   mem_prot_key
108113a8   __CIOBUF_
108114c8   __TI_STATIC_BASE
108114c8   gpXMC_regs
108114cc   gpCGEM_regs
108114d0   gpBootCfgRegs
108114d4   gpPLLC_regs
108114d8   gpPSC_regs
108114dc   gpMSMC_regs
108114e0   gpGPIO_regs
108114e4   gpARM_regs
108114e8   gpCIC0_regs
108114ec   gpCIC1_regs
108114f0   gpCIC_regs
108114f4   gpEDMA_CC0_regs
108114f8   gpEDMA_CC1_regs
108114fc   gpEDMA_CC2_regs
10811500   gpEDMA_CC3_regs
10811504   gpEDMA_CC4_regs
10811508   gpEDMA_TC_0_0_regs
1081150c   gpEDMA_TC_0_1_regs
10811510   gpEDMA_TC_1_0_regs
10811514   gpEDMA_TC_1_1_regs
10811518   gpEDMA_TC_1_2_regs
1081151c   gpEDMA_TC_1_3_regs
10811520   gpEDMA_TC_2_0_regs
10811524   gpEDMA_TC_2_1_regs
10811528   gpEDMA_TC_2_2_regs
1081152c   gpEDMA_TC_2_3_regs
10811530   gpEDMA_TC_3_0_regs
10811534   gpEDMA_TC_3_1_regs
10811538   gpEDMA_TC_4_0_regs
1081153c   gpEDMA_TC_4_1_regs
10811540   gARM_Core_Speed_Hz
10811544   gMain_Core_Speed_Hz
10811548   cycle_measure_overhead
1081154c   uiLL2_scrub_addr
10811550   LL2_EDC_victim_err_str
10811554   LL2_EDC_DMA_err_str
10811558   LL2_EDC_L1D_err_str
1081155c   LL2_EDC_L1P_err_str
10811560   guwIntcCICExcEvtIdx
10811564   gCIC_EXC_out_num
10811568   num_GPIO
1081156c   uiGPIO_host_event_num
1081198c   __TI_Handler_Table_Base
10811994   __TI_CINIT_Base
10811994   __TI_Handler_Table_Limit
108119ac   __TI_CINIT_Limit
ffffffff   __TI_pprof_out_hndl
ffffffff   __TI_prof_data_size
ffffffff   __TI_prof_data_start
ffffffff   __binit__
ffffffff   __c_args__
ffffffff   binit
UNDEFED    __TI_INITARRAY_Base
UNDEFED    __TI_INITARRAY_Limit
UNDEFED    __TI_TLS_INIT_Base
UNDEFED    __TI_TLS_INIT_Limit

[249 symbols]
